:020000040000FA
:02000000752B5E
:08000800A8000308A900040888
:10001000AA0083120C10FC308F0026308E000030B6
:100020008A00410882074C282B282D283028512887
:100030002B282D2833285628372839283B284C28A8
:100040003D283F284128512843284528472856283D
:10005000632863285B28CA206328CC30D720632814
:100060004430D7206328C001BE30D7206328042144
:100070006328092163280E2163281321632818218E
:1000800063281D21632822216328272163282C212E
:10009000CA10031DCA146328C3014508A3000A221D
:1000A0006328C30A4608A3000A226328C30A470834
:1000B000A3000A226328A20B63281430A2006E203A
:1000C000B12031226328C10A4108183A0319C1013D
:1000D000290883002A08840028080900B81D76280A
:1000E00038080739AB003708AC007B283808AB006C
:1000F000AB153708AC003608AC0735080318350FC8
:10010000AB07320834023108031C310F3302CE1022
:10011000031CCE143108CE183308A5003208CE18BF
:100120003408A6006E23031CCE153308CE18310800
:10013000A5003408CE183208A6006E230318CE118D
:10014000CE18A828CE1DA6284E16AE284E12AE28D0
:10015000CE19AC284E16AE284E12AE284A184E12B2
:10016000080030082C022F08031C2F0F2B02031845
:10017000BD282B08AF002C08B0002C082E022B083D
:10018000031C2B0F2D020318C9282B08AD002C08C7
:10019000AE00080005117630312100000515103041
:1001A00031214A1005194A14653031210800A30095
:1001B0000830A0000511DC28DD2823180515A30C44
:1001C000E128E228E328A3130519A3170C303121F5
:1001D0000515A00BDA2823080800A8000830A000A5
:1001E00028084006A300230C40080318183AA3006F
:1001F000230CC0000310A80C2808A00BF12808004D
:10020000C001BE30D7200800FF30D720B700ED2056
:100210000800FF30D720B800ED200800FF30D720BD
:10022000B900ED200800FF30D720BA00ED2008000B
:10023000FF30D720BB00ED200800FF30D720BC00E6
:10024000ED200800FF30D720BD00ED200800FF3072
:10025000D720BE00ED200800FF30D720BF00C0022D
:100260000800A1006400A10B32290800260E260711
:100270000F398318163E8318063E063E831CFA3E4D
:10028000261A1B3E831CFA3EA61A303E261B603EF1
:10029000A61B203E603EC801C80D481CA03EC900F8
:1002A00066302518BC30C9070318C80A0301031CAF
:1002B0006038831C0638C9026630A5187830C90733
:1002C0000318C80A0301031C6038831C0638C902DE
:1002D000260D250DA518013EC8070800480803197A
:1002E0000B30C7004908490E0F39031D7D29C80886
:1002F000031D7D29C90803190B30C60049080F39B1
:10030000C500080064008B1383161C1555309D0032
:10031000AA309D009C149C188B291C1583128C13E9
:1003200008000130CD00AB19AC294E15AB09AC0962
:10033000AC0A0318AC0A0319AC0A0730AB05A501D7
:10034000A030A6006E23031CBD292B08A5002C0895
:10035000A6000330CD00D2294E11AB11AF290630D3
:10036000A5004030A6006E23031CBD292B08A50064
:100370002C08A6000330CD00D2292B08A5002C089C
:10038000A6000330A0000310A60DA50DA00BC329E5
:100390000230A0002C08A6072B080318A50AA50701
:1003A000A00BCA290430A0000310A50CA60CA00BBA
:1003B000D42936216E214E1DE62946080B3A031D2D
:1003C000E4290F30C600E6290F30C70008000708EF
:1003D000A4000301051087128316051487168312E3
:1003E0000518CB14871A4B14831605108712831235
:1003F0002408870008000830A0000510A30C03188B
:100400000514871600008712A00BFD2907160000AF
:10041000071208000708F839A40003014E18073036
:1004200007392404870003308A002308DD23A30052
:1004300043084D06031D1D2AA3114E18A309FB21D5
:1004400022220800CC080319272A221E302A43083A
:10045000F223A3004E18A3090730230524048700C4
:100460000800E7214B080739A30002308A0023085F
:1004700082071A2BEB2A152B152B1A2B1A2B1A2B4A
:100480001A2B02308A0023084C0882071A2B4C2AA8
:100490004F2A36308400522A32308400522A3430B7
:1004A0008400522AC20A0130A0004208083A031D03
:1004B0005D2A0730C2000830A0000008A6008403AF
:1004C0000008A500A60F652AA50A4C08033A0319DF
:1004D000772A0F302502031C772A031D732AD03098
:1004E0002602031C772A0430A5009030A600A00B3A
:1004F000622A25088000840A260880000008A600D9
:1005000084030008A5001B2BCC011A2B02308A00A3
:100510004C0882071A2B902A932A36308400962A98
:1005200032308400962A34308400962AC20A013080
:10053000A0004208083A031DA12A0730C200083073
:10054000A0000008A60084030008A500A603260852
:10055000FF3A0319A5034C08033A0319BB2A2608DE
:10056000903C25080318250B043C031CBB2A0F30C4
:10057000A500D030A600A00BA62A25088000840A7A
:10058000260880000008A60084030008A5001B2B95
:100590000F30C2003230A200CC0A4C08043A0319D2
:1005A000D52A4C08033A031D1B2BCC01A001640083
:1005B0003130200784000008A300200883169B0028
:1005C00023089A0083128221A00A2008063A031DFC
:1005D000D72A8B171B2BC20A4208043A031D1B2B78
:1005E000C2012B08AD00AF002C08AE00B0001030E7
:1005F000C7000F30C6001130C5006D2B0D2B093020
:10060000B100B3009030B200B030B40082210F309E
:10061000C500C600C700C2016D2B42080E3A031D7B
:100620001B2BC2010330CC001B2BC408031D1A2B4B
:100630000630C400C201CC080319202B4B15212B16
:100640004B11CB104B1003308A004C0882072B2B28
:100650004A2B502B2B2BC4080319322B2830A20015
:10066000C4033C2B4A1C3C2B0E30C7001330C60081
:10067000C5000330CD006D2B4418632B2B30840054
:100680000310440884070008AB00840A0008AC008B
:100690009121562B3108AB003208AC009121562B2A
:1006A0003308AB003408AC009121562B42080F3AB6
:1006B000031D6D2B0330CD000F30C700C5004C0863
:1006C000F623C6006D2B0330CD001030C70011306B
:1006D000C500440CFA23C600CB01080026082C02F2
:1006E0002508031C250F2B0208008316FF2390000A
:1006F0008312850187018316CF3081008312C030B9
:100700008B000130900083169101850187019501CE
:100710008312073099002030A200223084003D303F
:10072000A0008001840AA003031D912B83160C14E2
:1007300083128F018E010430AD009030AE000F3077
:10074000AF00D030B0000130A20005154E144E129B
:10075000CA20CC30D7204E30D7200301D720030148
:10076000D7207F30D720831620089B001C141A083E
:10077000A300831203308A0020088207C42BC72BF2
:10078000CA2BCD2BD02BD32B2308B100D62B23087B
:10079000B200D62B2308B300D62B2308B400D62BE7
:1007A0002308B500D62B2308B600D62BA00A2008B4
:1007B000063A031DB32B6400DB2B820709346F3428
:1007C00058344A342E348A3488344F3408340A3446
:1007D0000C34FF3429342C349834FE3499344B349F
:1007E0001E34FC348207013402340434820703349B
:0C07F0000D3408348207123408340D3434
:02400E002C3F45
:0C420000080000000800000000000000A2
:00000001FF
